:020000040000FA
:04080000D8EF06F037
:1008100003B20AEF05F0F2B425EF05F09EB02DEF1C
:1008200005F09EB235EF05F0F2A81AEF04F0F2B22F
:100830001CEF04F087EF06F0CD90F2929EA026EF19
:1008400004F00101533F26EF04F0542BAEC1B2F186
:10085000AFC1B3F1B0C1B4F1B1C1B5F1AAC1AEF14C
:10086000ABC1AFF1ACC1B0F1ADC1B1F1A6C1AAF15C
:10087000A7C1ABF1A8C1ACF1A9C1ADF1A2C1A6F16C
:10088000A3C1A7F1A4C1A8F1A5C1A9F19EC1A2F17C
:100890009FC1A3F1A0C1A4F1A1C1A5F19AC19EF18C
:1008A0009BC19FF19CC1A0F19DC1A1F196C19AF19C
:1008B00097C19BF198C19CF199C19DF1CECF96F162
:1008C000CFCF97F153C198F154C199F1CF6ACE6A55
:1008D0000101536B546B9E90CD800FBC0F8E0FBAED
:1008E00075EF04F00F8A87EF06F00F8C0FBEB1EFA3
:1008F00004F096C19AF197C19BF198C19CF199C1FE
:100900009DF19AC19EF19BC19FF19CC1A0F19DC137
:10091000A1F19EC1A2F19FC1A3F1A0C1A4F1A1C107
:10092000A5F1A2C1A6F1A3C1A7F1A4C1A8F1A5C1D7
:10093000A9F1A6C1AAF1A7C1ABF1A8C1ACF1A9C1A7
:10094000ADF1AAC1AEF1ABC1AFF1ACC1B0F1ADC177
:10095000B1F1AEC1B2F1AFC1B3F1B0C1B4F1B1C147
:10096000B5F101015E6B5F6B606B616B96515E2749
:1009700097515F2398516023995161239A515E27C3
:100980009B515F239C5160239D5161239E515E27A3
:100990009F515F23A0516023A1516123A2515E2783
:1009A000A3515F23A4516023A5516123A6515E2763
:1009B000A7515F23A8516023A9516123AA515E2743
:1009C000AB515F23AC516023AD516123AE515E2723
:1009D000AF515F23B0516023B1516123B2515E2703
:1009E000B3515F23B4516023B5516123D890010105
:1009F000613360335F335E33D8900101613360331C
:100A00005F335E33D8900101613360335F335E330F
:100A100087EF06F00392030103EE00F080517F0B95
:100A2000E92604C0EFFF802B8151805D700BD8A4B4
:100A30008B8200008051815D700BD8A48B92815114
:100A40008019D8B4079087EF06F0F2940101453F72
:100A500087EF06F0462B87EF06F09E900101533F8B
:100A600087EF06F0542B87EF06F09E92C3CF55F127
:100A7000C4CF56F1C28207B4A0EF05F047C14BF1D5
:100A800048C14CF149C14DF14AC14EF15EC162F11C
:100A90005FC163F160C164F161C165F196C1B6F1F6
:100AA00097C1B7F198C1B8F199C1B9F19AC1BAF13A
:100AB0009BC1BBF19CC1BCF19DC1BDF19EC1BEF10A
:100AC0009FC1BFF1A0C1C0F1A1C1C1F1A2C1C2F1DA
:100AD000A3C1C3F1A4C1C4F1A5C1C5F1A6C1C6F1AA
:100AE000A7C1C7F1A8C1C8F1A9C1C9F1AAC1CAF17A
:100AF000ABC1CBF1ACC1CCF1ADC1CDF1AEC1CEF14A
:100B0000AFC1CFF1B0C1D0F1B1C1D1F1B2C1D2F119
:100B1000B3C1D3F1B4C1D4F1B5C1D5F1010155517F
:100B20005B2756515C23E86A5D230E2EA0EF05F08B
:100B30005CC157F15DC158F15B6B5C6B5D6B078EFF
:100B40000201002F87EF06F03C0E006F00C10CF190
:100B500001C10DF102C10EF103C10FF104C110F189
:100B600005C111F106C112F107C113F108C114F159
:100B700009C115F10AC116F10BC117F134C135F1E4
:100B800001018A67CBEF05F08B67CBEF05F08C672F
:100B9000CBEF05F08D67CFEF05F0FFEF05F08EC1CD
:100BA00000F18FC101F190C102F191C103F1010186
:100BB000010E046F000E056F000E066F000E076F2A
:100BC0001AEC15F000C18EF101C18FF102C190F154
:100BD00003C191F10067F4EF05F00167F4EF05F050
:100BE0000267F4EF05F00367FFEF05F08AC18EF1AD
:100BF0008BC18FF18CC190F18DC191F10F80D57EA9
:100C0000D5BE69D0D6CF47F1D7CF48F145C149F11C
:100C1000E86AE8CF4AF1109047C100F148C101F1FC
:100C200049C102F14AC103F101010A0E046F000E2D
:100C3000056F000E066F000E076F1AEC15F003AF7C
:100C40001080010154A731EF06F00F9A0F9C0F9E00
:100C50000101000E5E6F600E5F6F3D0E606F080E4B
:100C6000616F010147BF41EF06F0486741EF06F0B1
:100C7000496741EF06F04A6741EF06F0F28866EFF8
:100C800006F0F2985E6B5F6B606B616B966B976BB7
:100C9000986B996B9A6B9B6B9C6B9D6B9E6B9F6B20
:100CA000A06BA16BA26BA36BA46BA56BA66BA76BD0
:100CB000A86BA96BAA6BAB6BAC6BAD6BAE6BAF6B80
:100CC000B06BB16BB26BB36BB46BB56BD76AD66AF2
:100CD0000101456B466B0CC100F10DC101F10EC164
:100CE00002F10FC103F110C104F111C105F112C1EC
:100CF00006F113C107F114C108F115C109F116C1BC
:100D00000AF117C10BF135C134F187EF06F002C0CB
:100D1000E0FF005001C0D8FF1000A6B28DEF06F032
:100D20000CC0A9FF0BC0A8FFA69EA69CA684F29E9D
:100D3000550EA76EAA0EA76EA682F28EA694A6B234
:100D40009FEF06F00C2A1200A96EA69EA69CA68014
:100D5000A8500C2A120004012C0E826F8CEC08F0B3
:100D600015EC16F00C50A4EC06F0E8CF00F10C5096
:100D7000A4EC06F0E8CF01F101AFC4EF06F00101E9
:100D8000FF0E026FFF0E036FB8EC15F02967D0EF6E
:100D900006F00401200E826F8CEC08F0D5EF06F00F
:100DA00004012D0E826F8CEC08F0E2EC13F01200BF
:100DB000076A0F6A106A0F010E0EC16E860EC06EB2
:100DC000030EC26E0F01896A190E926E080E8A6EAA
:100DD000F10E936E8B6A800E946EF18E0E6A010195
:100DE0005B6B5C6B5D6B576B586BF29A0101476BE9
:100DF000486B496B4A6B4B6B4C6B4D6B4E6B4F6B3F
:100E0000506B516B526B456B466BD76AD66A0F01BC
:100E1000280ED56EF28A9D90B00ECD6E01015E6BEC
:100E20005F6B606B616B626B636B646B656B666B56
:100E3000676B686B696B536B546BCF6ACE6A0F9AA2
:100E40000F9C0F9E9D80760ECA6E9D8202013C0E05
:100E5000006FCC6A160EA4EC06F0E8CF00F1170E76
:100E6000A4EC06F0E8CF01F1180EA4EC06F0E8CFF0
:100E700002F1190EA4EC06F0E8CF03F1010103AF73
:100E80005CEF07F015EC16F0160E0C6E00C10BF0BF
:100E90008DEC06F0170E0C6E01C10BF08DEC06F018
:100EA000180E0C6E02C10BF08DEC06F0190E0C6ED4
:100EB00003C10BF08DEC06F000C18AF101C18BF18A
:100EC00002C18CF103C18DF100C18EF101C18FF11E
:100ED00002C190F103C191F11A0EA4EC06F0E8CF23
:100EE00000F11B0EA4EC06F0E8CF01F11C0EA4ECFF
:100EF00006F0E8CF02F11D0EA4EC06F0E8CF03F1F6
:100F0000010103AFB2EF07F015EC16F01A0E0C6EEC
:100F100000C10BF08DEC06F01B0E0C6E01C10BF046
:100F20008DEC06F01C0E0C6E02C10BF08DEC06F081
:100F30001D0E0C6E03C10BF08DEC06F01A0EA4EC26
:100F400006F0E8CF00F11B0EA4EC06F0E8CF01F1AB
:100F50001C0EA4EC06F0E8CF02F11D0EA4EC06F086
:100F6000E8CF03F100C192F101C193F102C194F104
:100F700003C195F1240EAC6E900EAB6E240EAC6ED8
:100F8000080EB86E80B6E3EF07F01E0EA4EC06F074
:100F9000E8CF00F11F0EA4EC06F0E8CF01F100C18C
:100FA000E8FFFF0A10E001C1E8FFFF0A0CE01E0E97
:100FB000A4EC06F0E8CFAFFF1F0EA4EC06F0E8CFDC
:100FC000B0FFE7EF07F0000EB06E1F0EAF6E04012A
:100FD000806B816B0F01900EAB6E0F019D8A030138
:100FE000806B816BC26B8B9207900001F28EF28C4A
:100FF00007B092EF12F00FB073EF0DF003018051C4
:1010000081197F0BD8B492EF12F013EE00F08151EA
:101010007F0BE126812BE7CFE8FFE00BD8B492EFFE
:1010200012F023EE82F0C2513F0BD926E7CFDFFF4B
:10103000C22BDF50780AD8A492EF12F007808EC13D
:1010400000F18FC101F190C102F191C103F10101E1
:10105000040E046F000E056F000E066F000E076F82
:101060001AEC15F000AF3EEF08F00101030E8E6F91
:10107000000E8F6F000E906F000E916F0301825172
:10108000720AD8B473EF0DF08251520AD8B473EFDC
:101090000DF08251750AD8B473EF0DF08251630AD6
:1010A000D8B44EEF0FF08251690AD8B431EF0AF08C
:1010B00082517A0AD8B444EF0BF08251490AD8B46D
:1010C000D0EF09F08251500AD8B4EEEF08F0825107
:1010D000700AD8B431EF09F08251540AD8B45CEFE9
:1010E00009F08251740AD8B4A2EF09F08251730A50
:1010F000D8B4A3EF0CF08251530AD8B408EF0DF026
:101100008251620AD8B4A0EF08F08251420AD8B4E2
:10111000DBEF08F083EF0FF0040114EE00F08051D4
:101120007F0BE12682C4E7FF802B120004010D0E25
:10113000826F8CEC08F00A0E826F8CEC08F01200C3
:101140008351610AD8A483EF0FF08451750AD8A4A3
:1011500083EF0FF08551640AD8A483EF0FF086C3A4
:101160002AF187C32BF188C32CF189C32DF18AC3DF
:101170002EF18BC32FF18CC330F18DC331F18EC3AF
:1011800032F18FC333F10101296B63EC16F0DAEC15
:1011900015F000C1AFFF01C1B0FF1E0E0C6EAFCF46
:1011A0000BF08DEC06F01F0E0C6EB0CF0BF08DEC3B
:1011B00006F083EF0FF080B6E5EF08F00401300E83
:1011C000826F8CEC08F0EAEF08F00401310E826FB8
:1011D0008CEC08F096EC08F083EF0FF083C32AF153
:1011E00084C32BF185C32CF186C32DF187C32EF167
:1011F00088C32FF189C330F18AC331F18BC332F137
:101200008CC333F1010163EC16F0DAEC15F0160E25
:101210000C6E00C10BF08DEC06F0170E0C6E01C1C8
:101220000BF08DEC06F0180E0C6E02C10BF08DEC7D
:1012300006F0190E0C6E03C10BF08DEC06F000C128
:101240008AF101C18BF102C18CF103C18DF100C1A2
:101250008EF101C18FF102C190F103C191F1D0EF84
:1012600009F083C32AF184C32BF185C32CF186C313
:101270002DF187C32EF188C32FF189C330F18AC3C2
:1012800031F18BC332F18CC333F1010163EC16F001
:10129000DAEC15F000C18AF101C18BF102C18CF1C9
:1012A00003C18DF100C18EF101C18FF102C190F136
:1012B00003C191F1D0EF09F083C32AF184C32BF16C
:1012C00085C32CF186C32DF187C32EF188C32FF17E
:1012D00089C330F18AC331F18CC332F18DC333F14C
:1012E000010163EC16F0DAEC15F00101000E046F59
:1012F000000E056F010E066F000E076F2BEC15F048
:101300001A0E0C6E00C10BF08DEC06F01B0E0C6E6D
:1013100001C10BF08DEC06F01C0E0C6E02C10BF03F
:101320008DEC06F01D0E0C6E03C10BF08DEC06F07B
:1013300000C192F101C193F102C194F103C195F191
:10134000D0EF09F083C32AF184C32BF185C32CF1BC
:1013500086C32DF187C32EF188C32FF189C330F1E5
:101360008AC331F18CC332F18DC333F1010163ECD7
:1013700016F0DAEC15F00101000E046F000E056F97
:10138000010E066F000E076F2BEC15F000C192F1F5
:1013900001C193F102C194F103C195F1D0EF09F0BD
:1013A000160EA4EC06F0E8CF00F1170EA4EC06F040
:1013B000E8CF01F1180EA4EC06F0E8CF02F1190E07
:1013C000A4EC06F0E8CF03F1B8EC15F09BEC13F0B9
:1013D0000401730E826F8CEC08F004012C0E826FF6
:1013E0008CEC08F08AC100F18BC101F18CC102F1D3
:1013F0008DC103F1B8EC15F09BEC13F00401730EF2
:10140000826F8CEC08F004012C0E826F8CEC08F0DB
:101410001A0EA4EC06F0E8CF00F11B0EA4EC06F0C7
:10142000E8CF01F11C0EA4EC06F0E8CF02F11D0E8E
:10143000A4EC06F0E8CF03F19EEC0FF004012C0EB3
:10144000826F8CEC08F092C100F193C101F194C15C
:1014500002F195C103F19EEC0FF096EC08F083EFDA
:101460000FF00401690E826F8CEC08F004012C0E61
:10147000826F8CEC08F00101040E006F000E016F0A
:10148000000E026F000E036FB8EC15F02CC182F451
:101490000401300E82278CEC08F02DC182F4040187
:1014A000300E82278CEC08F02EC182F40401300E3D
:1014B00082278CEC08F02FC182F40401300E8227C1
:1014C0008CEC08F030C182F40401300E82278CECE1
:1014D00008F031C182F40401300E82278CEC08F050
:1014E00032C182F40401300E82278CEC08F033C143
:1014F00082F40401300E82278CEC08F004012C0EDB
:10150000826F8CEC08F00101050E006F000E016F78
:10151000000E026F000E036FB8EC15F02CC182F4C0
:101520000401300E82278CEC08F02DC182F40401F6
:10153000300E82278CEC08F02EC182F40401300EAC
:1015400082278CEC08F02FC182F40401300E822730
:101550008CEC08F030C182F40401300E82278CEC50
:1015600008F031C182F40401300E82278CEC08F0BF
:1015700032C182F40401300E82278CEC08F033C1B2
:1015800082F40401300E82278CEC08F004012C0E4A
:10159000826F8CEC08F001011D0E006F000E016FD0
:1015A000000E026F000E036FB8EC15F02CC182F430
:1015B0000401300E82278CEC08F02DC182F4040166
:1015C000300E82278CEC08F02EC182F40401300E1C
:1015D00082278CEC08F02FC182F40401300E8227A0
:1015E0008CEC08F030C182F40401300E82278CECC0
:1015F00008F031C182F40401300E82278CEC08F02F
:1016000032C182F40401300E82278CEC08F033C121
:1016100082F40401300E82278CEC08F004012C0EB9
:10162000826F8CEC08F0200EF86EF76AF66A0401FF
:101630000900F5CF82F48CEC08F00900F5CF82F4B4
:101640008CEC08F00900F5CF82F48CEC08F009006E
:10165000F5CF82F48CEC08F00900F5CF82F48CEC25
:1016600008F00900F5CF82F48CEC08F00900F5CF02
:1016700082F48CEC08F00900F5CF82F48CEC08F0D1
:1016800096EC08F083EF0FF08351630AD8A483EF40
:101690000FF08451610AD8A483EF0FF085516C0AD2
:1016A000D8A483EF0FF08651410A3FE08651440AE7
:1016B0001BE08651420AD8B4A8EF0BF08651350AD8
:1016C000D8B40DEF11F08651360AD8B462EF11F09C
:1016D0008651370AD8B4CBEF11F08651380AD8B406
:1016E00029EF12F083EF0FF00798079A04017A0EA2
:1016F000826F8CEC08F00401780E826F8CEC08F09D
:101700000401640E826F8CEC08F00401550E826FA8
:101710008CEC08F091EF0BF004014C0E826F8CEC16
:1017200008F096EC08F083EF0FF00788079A0401A1
:101730007A0E826F8CEC08F00401410E826F8CEC03
:1017400008F00401610E826F8CEC08F085EF0BF05D
:101750000798078A04017A0E826F8CEC08F0040166
:10176000420E826F8CEC08F00401610E826F8CECEB
:1017700008F085EF0BF001016667C6EF0BF06767B5
:10178000C6EF0BF06867C6EF0BF06967DEEF0BF092
:101790004F67D2EF0BF05067D2EF0BF05167D2EFEB
:1017A0000BF05267DEEF0BF00101000E006F000E30
:1017B000016F000E026F000E036F12000101620E36
:1017C000046F010E056F000E066F000E076F66C1F5
:1017D00000F167C101F168C102F169C103F11AECBE
:1017E00015F003BF62EF0CF00101000E046FA80EAC
:1017F000056F550E066F020E076F66C100F167C1D7
:1018000001F168C102F169C103F166C186F167C1E6
:1018100087F168C188F169C189F11AEC15F003BF3D
:101820001BEF0CF00101000E866FA80E876F550E9E
:10183000886F020E896F0E0EA4EC06F0E8CF18F147
:101840000F0EA4EC06F0E8CF19F1100EA4EC06F090
:10185000E8CF1AF1110EA4EC06F0E8CF1BF163EC0F
:1018600014F086C104F187C105F188C106F189C170
:1018700007F11AEC15F0078227EC14F063EC14F072
:10188000079227EC14F086C100F187C101F188C1ED
:1018900002F189C103F1079227EC14F0CC0E046F1A
:1018A000E00E056F870E066F050E076F1AEC15F038
:1018B00000C118F101C119F102C11AF103C11BF1F4
:1018C0009AEF0CF00101800E006F1A0E016F060EE8
:1018D000026F000E036F4FC104F150C105F151C1F9
:1018E00006F152C107F11AEC15F003AF7BEF0CF0D3
:1018F00015EC16F012000E0EA4EC06F0E8CF18F16D
:101900000F0EA4EC06F0E8CF19F1100EA4EC06F0CF
:10191000E8CF1AF1110EA4EC06F0E8CF1BF14FC18D
:1019200000F150C101F151C102F152C103F107822E
:1019300027EC14F018C100F119C101F11AC102F12C
:101940001BC103F112000401730E826F8CEC08F0CE
:1019500004012C0E826F8CEC08F0078462C166F1E2
:1019600063C167F164C168F165C169F14BC14FF1B1
:101970004CC150F14DC151F14EC152F157C159F115
:1019800058C15AF10794C9EC0CF096EC08F083EFBB
:101990000FF066C100F167C101F168C102F169C1D0
:1019A00003F10101B8EC15F09BEC13F00401630E98
:1019B000826F8CEC08F004012C0E826F8CEC08F026
:1019C0004FC100F150C101F151C102F152C103F107
:1019D0000101B8EC15F09BEC13F00401660E826F68
:1019E0008CEC08F004012C0E826F8CEC08F015ECE6
:1019F00016F059C100F15AC101F10101B8EC15F01E
:101A00009BEC13F00401740E826F8CEC08F0120052
:101A100010820401530E826F8CEC08F004012C0E2E
:101A2000826F8CEC08F083C32AF184C32BF185C349
:101A30002CF186C32DF187C32EF188C32FF189C302
:101A400030F18AC331F18BC332F18CC333F1010120
:101A500063EC16F0DAEC15F000C166F101C167F134
:101A600002C168F103C169F18EC32AF18FC32BF162
:101A700090C32CF191C32DF192C32EF193C32FF19A
:101A800094C330F195C331F196C332F197C333F16A
:101A9000010163EC16F0DAEC15F000C14FF101C161
:101AA00050F102C151F103C152F156EC16F099C345
:101AB0002FF19AC330F19BC331F19CC332F19DC326
:101AC00033F1010163EC16F0DAEC15F000C159F1C5
:101AD00001C15AF1C9EC0CF004012C0E826F8CECA0
:101AE00008F07AEF0DF08251520A03E10F827AEF8B
:101AF0000DF00F928251750A03E1108481EF0DF011
:101B000010948251550A03E1108688EF0DF010966B
:101B1000078410B2E5EF0DF010A4D1EF0DF0B6C1BF
:101B200066F1B7C167F1B8C168F1B9C169F1BAC16D
:101B30006AF1BBC16BF1BCC16CF1BDC16DF1BEC13D
:101B40006EF1BFC16FF1C0C170F1C1C171F1C2C10D
:101B500072F1C3C173F1C4C174F1C5C175F1C6C1DD
:101B600076F1C7C177F1C8C178F1C9C179F1CAC1AD
:101B70007AF1CBC17BF1CCC17CF1CDC17DF1CEC17D
:101B80007EF1CFC17FF1D0C180F1D1C181F1D2C14D
:101B900082F1D3C183F1D4C184F1D5C185F1D9EFEC
:101BA0000DF062C166F163C167F164C168F165C19E
:101BB00069F14BC14FF14CC150F14DC151F14EC1D2
:101BC00052F157C159F158C15AF107940FA007EFCC
:101BD0000EF001019267F4EF0DF09367F4EF0DF052
:101BE0009467F4EF0DF09567F8EF0DF007EF0EF046
:101BF000BBEC0BF092C104F193C105F194C106F165
:101C000095C107F11AEC15F003BF4BEF0FF0BBECD9
:101C10000BF00101000E046F000E056F010E066F40
:101C2000000E076F4BEC15F010A41EEF0EF0040130
:101C3000750E826F8CEC08F023EF0EF00401720E2B
:101C4000826F8CEC08F004012C0E826F8CEC08F093
:101C5000B8EC15F0296732EF0EF00401200E826F08
:101C600035EF0EF004012D0E826F8CEC08F030C1C0
:101C700082F40401300E82278CEC08F031C182F42A
:101C80000401300E82278CEC08F004012E0E826FC6
:101C90008CEC08F032C182F40401300E82278CEC07
:101CA00008F033C182F40401300E82278CEC08F076
:101CB00004016D0E826F8CEC08F004012C0E826F13
:101CC0008CEC08F04FC100F150C101F151C102F19B
:101CD00052C103F10101B8EC15F09BEC13F00401C3
:101CE000480E826F8CEC08F004017A0E826F8CEC47
:101CF00008F004012C0E826F8CEC08F066C100F134
:101D000067C101F168C102F169C103F10101B8ECD9
:101D100015F09BEC13F00401630E826F8CEC08F05D
:101D200004012C0E826F8CEC08F066C100F167C1D3
:101D300001F168C102F169C103F101010A0E046FEA
:101D4000000E056F000E066F000E076F2BEC15F0EE
:101D5000000E046F120E056F000E066F000E076F67
:101D60004BEC15F0B8EC15F02AC182F40401300EEA
:101D700082278CEC08F02BC182F40401300E8227FC
:101D80008CEC08F02CC182F40401300E82278CEC1C
:101D900008F02DC182F40401300E82278CEC08F08B
:101DA0002EC182F40401300E82278CEC08F02FC182
:101DB00082F40401300E82278CEC08F030C182F4EA
:101DC0000401300E82278CEC08F004012E0E826F85
:101DD0008CEC08F031C182F40401300E82278CECC7
:101DE00008F032C182F40401300E82278CEC08F036
:101DF00033C182F40401300E82278CEC08F0040118
:101E0000730E826F8CEC08F004012C0E826F8CEC48
:101E100008F015EC16F059C100F15AC101F1ADEC12
:101E200010F00FB217EF0FF00FA049EF0FF0040101
:101E30002C0E826F8CEC08F0200EF86EF76AF66AB2
:101E400004010900F5CF82F48CEC08F00900F5CF0D
:101E500082F48CEC08F00900F5CF82F48CEC08F0E9
:101E60000900F5CF82F48CEC08F00900F5CF82F47C
:101E70008CEC08F00900F5CF82F48CEC08F0090036
:101E8000F5CF82F48CEC08F00900F5CF82F48CECED
:101E900008F096EC08F00F9083EF0FF00401630E4A
:101EA000826F8CEC08F004012C0E826F8CEC08F031
:101EB00089EC0FF004012C0E826F8CEC08F0FCEC26
:101EC0000FF004012C0E826F8CEC08F078EC10F00F
:101ED00004012C0E826F8CEC08F00101F80E006FEB
:101EE000CD0E016F660E026F030E036F9EEC0FF0B6
:101EF00004012C0E826F8CEC08F08EEC10F096EC46
:101F000008F083EF0FF00301C26B0790109292EF7D
:101F100012F0D8900E0EA4EC06F0E8CF00F10F0EF0
:101F2000A4EC06F0E8CF01F1100EA4EC06F0E8CF27
:101F300002F1110EA4EC06F0E8CF03F10101000E4E
:101F4000046F000E056F010E066F000E076F4BEC5D
:101F500015F0B8EC15F02AC182F40401300E822786
:101F60008CEC08F02BC182F40401300E82278CEC3B
:101F700008F02CC182F40401300E82278CEC08F0AA
:101F80002DC182F40401300E82278CEC08F02EC1A2
:101F900082F40401300E82278CEC08F02FC182F409
:101FA0000401300E82278CEC08F030C182F4040169
:101FB000300E82278CEC08F031C182F40401300E1F
:101FC00082278CEC08F004012E0E826F8CEC08F056
:101FD00032C182F40401300E82278CEC08F033C148
:101FE00082F40401300E82278CEC08F004016D0E9F
:101FF000826F8CEC08F01200120EA4EC06F0E8CF11
:1020000000F1130EA4EC06F0E8CF01F1140EA4ECDD
:1020100006F0E8CF02F1150EA4EC06F0E8CF03F1CC
:1020200001010A0E046F000E056F000E066F000E10
:10203000076F2BEC15F0000E046F120E056F000EEB
:10204000066F000E076F4BEC15F0B8EC15F02AC1C7
:1020500082F40401300E82278CEC08F02BC182F44C
:102060000401300E82278CEC08F02CC182F40401AC
:10207000300E82278CEC08F02DC182F40401300E62
:1020800082278CEC08F02EC182F40401300E8227E6
:102090008CEC08F02FC182F40401300E82278CEC06
:1020A00008F030C182F40401300E82278CEC08F075
:1020B00004012E0E826F8CEC08F031C182F4040111
:1020C000300E82278CEC08F032C182F40401300E0D
:1020D00082278CEC08F033C182F40401300E822791
:1020E0008CEC08F00401730E826F8CEC08F0120087
:1020F0000A0EA4EC06F0E8CF00F10B0EA4EC06F0FB
:10210000E8CF01F10C0EA4EC06F0E8CF02F10D0EC1
:10211000A4EC06F0E8CF03F1ADEF10F0060EA4EC4E
:1021200006F0E8CF00F1070EA4EC06F0E8CF01F1CD
:10213000080EA4EC06F0E8CF02F1090EA4EC06F0BC
:10214000E8CF03F1ADEF10F0010115EC16F00784B4
:1021500057C100F158C101F107940101E80E046F65
:10216000800E056F000E066F000E076F2BEC15F04A
:10217000000E046F040E056F000E066F000E076F51
:102180004BEC15F0880E046F130E056F000E066FF2
:10219000000E076F1AEC15F00A0E046F000E056FA3
:1021A000000E066F000E076F4BEC15F0B8EC15F043
:1021B00001012967E1EF10F00401200E826FE4EFC6
:1021C00010F004012D0E826F8CEC08F030C182F407
:1021D0000401300E82278CEC08F031C182F4040136
:1021E000300E82278CEC08F032C182F40401300EEC
:1021F00082278CEC08F004012E0E826F8CEC08F024
:1022000033C182F40401300E82278CEC08F0040103
:10221000430E826F8CEC08F0120087C32AF188C34A
:102220002BF189C32CF18AC32DF18BC32EF18CC302
:102230002FF18DC330F18EC331F190C332F191C3D0
:1022400033F10101296B63EC16F0DAEC15F00101B2
:10225000000E046F000E056F010E066F000E076F73
:102260002BEC15F00E0E0C6E00C10BF08DEC06F091
:102270000F0E0C6E01C10BF08DEC06F0100E0C6E03
:1022800002C10BF08DEC06F0110E0C6E03C10BF0C9
:102290008DEC06F004017A0E826F8CEC08F00401DC
:1022A0002C0E826F8CEC08F00401350E826F8CECE2
:1022B00008F004012C0E826F8CEC08F089EC0FF012
:1022C00091EF0BF087C32AF188C32BF189C32CF15E
:1022D0008AC32DF18BC32EF18CC32FF18DC330F146
:1022E0008EC331F190C332F191C333F10101296BF7
:1022F00063EC16F0DAEC15F0880E046F130E056F20
:10230000000E066F000E076F1FEC15F0000E046F35
:10231000040E056F000E066F000E076F2BEC15F014
:102320000101E80E046F800E056F000E066F000EAF
:10233000076F4BEC15F00A0E0C6E00C10BF08DEC24
:1023400006F00B0E0C6E01C10BF08DEC06F00C0EBE
:102350000C6E02C10BF08DEC06F00D0E0C6E03C17D
:102360000BF08DEC06F004017A0E826F8CEC08F015
:1023700004012C0E826F8CEC08F00401360E826F83
:102380008CEC08F004012C0E826F8CEC08F078ECD9
:1023900010F091EF0BF087C32AF188C32BF189C3AA
:1023A0002CF18AC32DF18BC32EF18CC32FF18DC379
:1023B00030F18FC331F190C332F191C333F1010198
:1023C00063EC16F0DAEC15F0000E046F120E056FD8
:1023D000000E066F000E076F2BEC15F001010A0EC0
:1023E000046F000E056F000E066F000E076F4BECBA
:1023F00015F0120E0C6E00C10BF08DEC06F0130EF2
:102400000C6E01C10BF08DEC06F0140E0C6E02C1C7
:102410000BF08DEC06F0150E0C6E03C10BF08DEC7D
:1024200006F004017A0E826F8CEC08F004012C0E89
:10243000826F8CEC08F00401370E826F8CEC08F090
:1024400004012C0E826F8CEC08F0FCEC0FF091EF85
:102450000BF087C32AF188C32BF189C32CF18AC3FF
:102460002DF18BC32EF18CC32FF18DC330F18EC3B0
:1024700031F190C332F191C333F10101296B63EC67
:1024800016F0DAEC15F0880E046F130E056F000ECF
:10249000066F000E076F1FEC15F0000E046F040EA0
:1024A000056F000E066F000E076F2BEC15F0010193
:1024B000E80E046F800E056F000E066F000E076FAA
:1024C0004BEC15F0060E0C6E00C10BF08DEC06F017
:1024D000070E0C6E01C10BF08DEC06F0080E0C6EB1
:1024E00002C10BF08DEC06F0090E0C6E03C10BF06F
:1024F0008DEC06F004017A0E826F8CEC08F004017A
:102500002C0E826F8CEC08F00401380E826F8CEC7C
:1025100008F004012C0E826F8CEC08F08EEC10F0A9
:1025200091EF0BF007A806EF13F00101800E006F8A
:102530001A0E016F060E026F000E036F4BC104F1FD
:102540004CC105F14DC106F14EC107F11AEC15F071
:1025500003BF4DEF13F095EC13F04BC100F14CC1EC
:1025600001F14DC102F14EC103F1078227EC14F0D5
:1025700018C104F119C105F11AC106F11BC107F117
:10258000F80E006FCD0E016F660E026F030E036F23
:102590001AEC15F00E0E0C6E00C10BF08DEC06F06F
:1025A0000F0E0C6E01C10BF08DEC06F0100E0C6ED0
:1025B00002C10BF08DEC06F0110E0C6E03C10BF096
:1025C0008DEC06F00784010115EC16F057C100F1FF
:1025D00058C101F107940A0E0C6E00C10BF08DEC8E
:1025E00006F00B0E0C6E01C10BF08DEC06F00C0E1C
:1025F0000C6E02C10BF08DEC06F00D0E0C6E03C1DB
:102600000BF08DEC06F007984DEF13F007AA4DEF95
:1026100013F00784010115EC16F057C100F158C101
:1026200001F10794060E0C6E00C10BF08DEC06F064
:10263000070E0C6E01C10BF08DEC06F0080E0C6E4F
:1026400002C10BF08DEC06F0090E0C6E03C10BF00D
:102650008DEC06F0078462C100F163C101F164C131
:1026600002F165C103F10794120E0C6E00C10BF06C
:102670008DEC06F0130E0C6E01C10BF08DEC06F024
:10268000140E0C6E02C10BF08DEC06F0150E0C6EE4
:1026900003C10BF08DEC06F0079A040180518119FB
:1026A0007F0B0BE09EA809D014EE00F081517F0B48
:1026B000E126E750812B0F01AD6EF8EF07F018C14E
:1026C00000F119C101F11AC102F11BC103F1000EA1
:1026D000046F000E056F010E066F000E076F4BECC6
:1026E00015F029A18AEF13F02051D8B48AEF13F026
:1026F00018C100F119C101F11AC102F11BC103F1A6
:10270000000E046F000E056F0A0E066F000E076FB5
:102710004BEC15F012000101045100130551011397
:10272000065102130751031312000101186B196BB4
:102730001A6B1B6B12002AC182F40401300E82272F
:102740008CEC08F02BC182F40401300E82278CEC53
:1027500008F02CC182F40401300E82278CEC08F0C2
:102760002DC182F40401300E82278CEC08F02EC1BA
:1027700082F40401300E82278CEC08F02FC182F421
:102780000401300E82278CEC08F030C182F4040181
:10279000300E82278CEC08F031C182F40401300E37
:1027A00082278CEC08F032C182F40401300E8227BB
:1027B0008CEC08F033C182F40401300E82278CECDB
:1027C00008F012002FC182F40401300E82278CEC35
:1027D00008F030C182F40401300E82278CEC08F03E
:1027E00031C182F40401300E82278CEC08F032C132
:1027F00082F40401300E82278CEC08F033C182F49D
:102800000401300E82278CEC08F01200060E116EC7
:10281000060E126E060E136E112E0CEF14F0122E11
:102820000CEF14F0132E0CEF14F08B84020E116ECB
:10283000020E126E020E136E112E1CEF14F0122EE9
:102840001CEF14F0132E1CEF14F08B9412000101F6
:10285000005305E1015303E1025301E1002BEAECCF
:1028600014F015EC16F03951006F3A51016F420E19
:10287000046F4B0E056F000E066F000E076F2BECFA
:1028800015F000C104F101C105F102C106F103C157
:1028900007F118C100F119C101F11AC102F11BC100
:1028A00003F107B258EF14F01FEC15F05AEF14F0D3
:1028B0001AEC15F000C118F101C119F102C11AF1A9
:1028C00003C11BF1120015EC16F059C100F15AC1F9
:1028D00001F1060EA4EC06F0E8CF04F1070EA4EC1B
:1028E00006F0E8CF05F1080EA4EC06F0E8CF06F1FB
:1028F000090EA4EC06F0E8CF07F11AEC15F000C1C0
:1029000024F101C125F102C126F103C127F1290EED
:10291000046F000E056F000E066F000E076F2BECA4
:1029200015F0EE0E046F430E056F000E066F000EDD
:10293000076F1FEC15F024C104F125C105F126C174
:1029400006F127C107F12BEC15F000C11CF101C104
:102950001DF102C11EF103C11FF1120EA4EC06F01D
:10296000E8CF04F1130EA4EC06F0E8CF05F1140E45
:10297000A4EC06F0E8CF06F1150EA4EC06F0E8CFC3
:1029800007F10D0E006F000E016F000E026F000EBA
:10299000036F2BEC15F0180E046F000E056F000E80
:1029A000066F000E076F4BEC15F01CC104F11DC142
:1029B00005F11EC106F11FC107F11FEC15F06A0EEB
:1029C000046F2A0E056F000E066F000E076F1AECDB
:1029D00015F01200BF0EFA6E200E3A6F396BD890C8
:1029E0000037013702370337D8B0FBEF14F03A2F26
:1029F000F0EF14F039073A070353D8B4120003314B
:102A0000070B80093F6F03390F0B010F396F80EC03
:102A10005FF0406F390580EC5FF0405D405F396BDF
:102A20003F33D8B0392739333FA910EF15F0405163
:102A30003927120001013AEC16F0D8B0120001015A
:102A400003510719346FFDEC15F0D89007510319A5
:102A500034AF800F12000101346B21EC16F0D8A0C6
:102A600037EC16F0D8B012000CEC16F015EC16F09E
:102A70001F0E366F4DEC16F00B35D8B0FDEC15F08F
:102A8000D8A00335D8B01200362F3AEF15F034B184
:102A900024EC16F012000101346B045105110611EB
:102AA00007110008D8A021EC16F0D8A037EC16F0DA
:102AB000D8B01200086B096B0A6B0B6B4DEC16F06B
:102AC0001F0E366F4DEC16F007510B5DD8A475EF55
:102AD00015F006510A5DD8A475EF15F00551095D92
:102AE000D8A475EF15F00451085DD8A088EF15F053
:102AF0000451085F0551D8A0053D095F0651D8A0D3
:102B0000063D0A5F0751D8A0073D0B5FD8900081B2
:102B1000362F62EF15F034B124EC16F0346B21EC53
:102B200016F0D89051EC16F007510B5DD8A4A5EF24
:102B300015F006510A5DD8A4A5EF15F00551095D01
:102B4000D8A4A5EF15F00451085DD8A0B4EF15F096
:102B5000003FB4EF15F0013FB4EF15F0023FB4EFC2
:102B600015F0032BD8B4120034B124EC16F0120087
:102B70000101346B21EC16F0D8B0120056EC16F0BF
:102B8000200E366F003701370237033711EE33F06E
:102B90000A0E376FE7360A0EE75CD8B0E76EE552EB
:102BA000372FCAEF15F0362FC2EF15F034B1298157
:102BB000D890120001010A0E346F200E366F11EE0C
:102BC00029F03451376F0A0ED890E652D8B0E72674
:102BD000E732372FE5EF15F00333023301330033CB
:102BE000362FDFEF15F0E750FF0FD8A00335D8B030
:102BF000120029B124EC16F01200045100270551EF
:102C0000D8B0053D01270651D8B0063D022707512F
:102C1000D8B0073D032712000051086F0151096F1A
:102C200002510A6F03510B6F12000101006B016B1F
:102C3000026B036B12000101046B056B066B076BE3
:102C400012000335D8A012000351800B001F011F92
:102C5000021F031F003F34EF16F0013F34EF16F060
:102C6000023F34EF16F0032B342B032512000735F7
:102C7000D8A012000751800B041F051F061F071F55
:102C8000043F4AEF16F0053F4AEF16F0063F4AEFC1
:102C900016F0072B342B07251200003701370237B7
:102CA0000337083709370A370B3712000101296B40
:102CB0002A6B2B6B2C6B2D6B2E6B2F6B306B316B50
:102CC000326B336B120001012A510F0B2A6F2B510B
:102CD0000F0B2B6F2C510F0B2C6F2D510F0B2D6FDA
:102CE0002E510F0B2E6F2F510F0B2F6F30510F0BDB
:102CF000306F31510F0B316F32510F0B326F335137
:062D00000F0B336F1200FF
:10BF0000E844F926000C160C2B0C3F0C520C640C68
:10BF1000760C860C960CA50CB30CC10CCF0CDC0C6B
:06BF2000E80CF40C000C1B
:00000001FF
